:020000040800F2
:10200000D82D0020292100083121000833210008A3
:1020100035210008372100083921000800000000A0
:102020000000000000000000000000003B2100084C
:102030003D210008000000003F2100082152000857
:1020400043210008C9420008432100084321000839
:10205000432100084321000861300008FD300008DA
:102060001D3100083D3100085D310008F9280008E5
:1020700043210008432100084321000835290008B6
:1020800043210008432100084321000843210008A0
:1020900043210008432100087D3100084321000846
:1020A000432100084321000843210008415400084F
:1020B00091540008E554000843210008432100081A
:1020C0000D3E0008993D0008432100084321000807
:1020D0004321000843210008432100088130000803
:1020E0004321000843210008432100084321000840
:1020F000432100084321000843210008315500080E
:1021000079550008432100084321000843210008B5
:1021100043210008DFF80CD000F07EF800480047AB
:10212000A1600008D82D00200648804706480047D7
:10213000FEE7FEE7FEE7FEE7FEE7FEE7FEE7FEE777
:10214000FEE7FEE7915300081521000840EA01036D
:102150009B0703D009E008C9121F08C0042AFAD25D
:1021600003E011F8013B00F8013B521EF9D2704721
:10217000D2B201E000F8012B491EFBD270470022C9
:10218000F6E710B513460A4604461946FFF7F0FF76
:10219000204610BD2DE9F05F0546002092469B4683
:1021A00088460646814640241BE02846414647466D
:1021B000224600F020F853465A46C01A914110D3E7
:1021C00011461846224600F039F82D1A67EB01082F
:1021D0004F4622460120002100F030F817EB00099D
:1021E0004E41201EA4F10104DFDC484631462A4658
:1021F0004346BDE8F09F202A04DB203A21FA02F092
:102200000021704721FA02F3D040C2F12002914030
:102210000843194670470000064C074D06E0E06889
:1022200040F0010394E8070098471034AC42F6D31D
:10223000FFF774FFB46E0008D46E0008202A04DB98
:10224000203A00FA02F1002070479140C2F12003C9
:1022500020FA03F319439040704700002DE9F04144
:102260000F004FF00002804605D0017801233C4E5C
:10227000302903D00DE00420BDE8F081C17821B100
:10228000012905D0022903D02CE00021317000E0A3
:1022900033700178102925D14178012922D1304CA1
:1022A0008178641DFF25112910D190F803C0BCF17D
:1022B000100F17D173701123B3700F232370657043
:1022C0000378102B0ED14378012B0BD1222909D191
:1022D000C178102906D1022171702221B170072125
:1022E00021706570C119057811F8014C1C49042D45
:1022F000CB782BD006DC012D28D0022D18D0032D51
:1023000006D115E0062D23D0302D1FD0902D01D001
:102310000120B1E701F0AAF903F0E2FB0120F0701F
:10232000AC4201D114E00BB10020F0700220A3E711
:1023300000217D1E05E010F801CB491C8CEA020249
:1023400089B2A942F7DB9442EDD101E0AC42EAD177
:102350007A1E41460348FFF7F9FE00208CE7000093
:1023600080000020680300208C498C4A2DE9F14F41
:1023700001F07041C2F3130201EB4212874984B0AD
:10238000CE3101F07043C1F3130103EB41138449D3
:10239000814801F07044C1F3130104EB41148049FA
:1023A0000290CE3101F07045C1F3130105EB4111EC
:1023B000443901F1007E7B49443A01F07045C1F394
:1023C000130105EB411577492020CE3101F070460D
:1023D000C1F3130106EB4111443901F10071009181
:1023E000714902F1007201F07046C1F3130106EB6E
:1023F0004111443901F1007A6B49CE3101F0704648
:10240000C1F3130106EB4116684901F07047C1F3AF
:10241000130107EB4111443901F1007B6349CE31CF
:1024200001F07047C1F3130107EB4111443901F189
:1024300000795949CE3901F07047C1F3130107EB18
:102440004111443901F1007101910021443B03F134
:102450000073443C443D443E04F1007405F10075B2
:1024600006F10076039190E0090719D1009902EB7B
:10247000800201EB80010091019903EB800301EBE5
:10248000800104EB80040EEB800E05EB80050AEB67
:10249000800A06EB80060BEB800B09EB80090191AB
:1024A000029900270F80424932F80479096991F8AE
:1024B00000C091F8018007FA0CF733F804C90CFA50
:1024C00008FC47EA0C0734F804C991F802800CFABA
:1024D00008FC47EA0C07BEF800C091F80380AEF193
:1024E000040E0CFA08FC47EA0C0735F804C991F809
:1024F00004800CFA08FC47EA0C07DDF800C091F8EC
:102500000580BCF800C00CFA08FC47EA0C07BAF8D2
:1025100000C091F80680AAF1040A0CFA08FC47EA08
:102520000C0736F804C991F807800CFA08FC47EA52
:102530000C07BBF800C091F80880ABF1040B0CFA53
:1025400008FC47EA0C07B9F800C091F80980897ABD
:102550000CFA08FC47EA0C07DDF804C0A9F10409ED
:10256000BCF800C00CFA01FC029947EA0C070F8086
:102570000299891C02910099091F00910199091F74
:1025800001910399491C89B20391049FB942FFF458
:102590006BAF05B0BDE8F08FD6180020FC0F00200F
:1025A0009811002034130020D01400206C16002055
:1025B000980F00207EB50025DDE90746ADF80050F4
:1025C0008DF804508DF80850ADF80030761E8DF867
:1025D00004601BE09DF8043020FA03F303F00103CC
:1025E0008DF808309DF80830002BBDF8003000D081
:1025F000634022F8023B9BB2634021F8023BADF8F6
:1026000000309DF804305B1E8DF804309DF90430D5
:10261000002BDFDABDF800007EBD00007CB5224D46
:10262000792119227A2002F0E5FC642003F006FDEE
:1026300040F6DA011D48FFF7A2FD1D4C40F6FF7180
:10264000608935F8100000F00F02C0F3061302EBAA
:10265000C302C00A672310FB03F0144B002503EBF1
:10266000400000EB42000122818112481146857032
:102670006020CDE900501048837A284602F0EAFC39
:102680000A2003F0C3FC608A401C80B260821428D8
:1026900008D165826089401C80B26081B0F5846F8A
:1026A00000D165817CBD000024620008FC0F002081
:1026B00002000020C6290020980F00202DE9FC41CF
:1026C000394C792119227A2002F094FC642003F01D
:1026D000B5FC40F6DA013548FFF751FD344D334A79
:1026E00040F6FF732E894FF000002C2E1CD200EB19
:1026F000400101EBC00106EB810134F8111001F03B
:102700000F07C1F3061C07EBCC07C90A4FF0670C93
:1027100011FB0CF102EB410101EB4701401C80B2BF
:102720008B811828E3D31FE006EB460101EBC606B8
:1027300000EB860104EB4101A1F58051B1F8E010F6
:1027400001F00F07C1F3061C07EBCC07C90A4FF0D5
:10275000670C11FB0CF102EB410101EB4701401C3E
:1027600080B28B812C28E3D312480024012284708C
:102770006020CDE9004010481146837A204602F0DF
:1027800069FC0A2003F042FC288A401C80B228829F
:10279000142807D12C822889401C80B22881442823
:1027A00000D12C81BDE8FC8124620008FC0F0020D0
:1027B00002000020C6290020980F00207CB51B488D
:1027C000002479210481448119227A2002F012FC2C
:1027D000642003F033FC40F6DA011548FFF7CFFC24
:1027E000134D002140F6FF72002067234B4305EB99
:1027F000430303EB4006401C80B2B2816028F8D34B
:10280000491C89B20B29EFD30A4801221146847072
:102810006020CDE900400848837A002002F01AFCCD
:10282000BDE87C40082003F0F1BB0000020000205E
:10283000FC0F0020C6290020980F00202DE9F04150
:1028400086B04FF4007001F02DFF4FF4806001F06E
:1028500029FF684601F05AF80125AF03124ECDE971
:102860000075002469463046039401F010F839469B
:10287000304601F036F8EE03DFF83080CDE9006530
:1028800069464046039401F002F83146404601F0A3
:1028900026F8CDE90145694640460097039400F0CB
:1028A000F6FF06B0BDE8F08100400240003C024067
:1028B000002204E030F8023B5A40491E89B2002948
:1028C000F8D1104670470000014900200870704799
:1028D000A6000020074B10B5002093F88320014686
:1028E000521E04E05C18A4786040491CC9B28A42B8
:1028F000F8DC10BD6A0500200B4810B50168890797
:1029000011D5416841F00F01416008480121017073
:10291000002141800448083000F02CF8BDE8104048
:10292000034801F0CEBF10BD00000240A600002009
:10293000003C01400C4810B50168890313D541687B
:1029400041F470214160094C206820F001002060B2
:102950006115204602F0E9FEA115204602F0E5FED1
:1029600003490020087410BD00000240000400402C
:10297000740E0020016821F00101016070470161BF
:102980007047026822F02002026002680A43026077
:102990007047026822F01002026002680A43026077
:1029A000704710B5044608680B46A0604868E060B0
:1029B00089682046FFF7EDFFD868606020461969F6
:1029C00000F032F82046596900F01EF82046996957
:1029D00000F032F82046D96900F01EF82046196A46
:1029E000FFF7CFFF2046596A00F02EF82046996A7B
:1029F000BDE81040AFF30080026822F4804202601C
:102A000002680A4302607047026822F08002026096
:102A100002680A4302607047026822F44062026062
:102A200002680A4302607047026822F040020260B6
:102A300002680A4302607047026822F44072026032
:102A400002680A4302607047026822F44052026042
:102A500002680A4302607047016821F001010160C9
:102A60000021016041608160C1602149204A08392C
:102A7000904203D1486840F00F0006E01C4A14322F
:102A8000904204D1486840F0F00048607047184A0E
:102A90002832904203D1486840F47060F5E7144A48
:102AA0003C32904203D1486840F47040EDE7104A50
:102AB0005032904203D1486840F47020E5E70C4A58
:102AC0006432904203D1486840F47000DDE7084A60
:102AD0007832904203D1486840F07060D5E7044AEC
:102AE0008C329042D2D1486840F07040CDE700006F
:102AF000080002400021016041608160C160016105
:102B000041618161C161016241628162704700007F
:102B10002DE9F047854F0025A7F2022301261978F9
:102B200039702C4603227E7018B1BA7087F8832062
:102B30008DE00026BE70DFF8F88187F88320994683
:102B40004FF4104A042928D004DC022926D0032996
:102B50007DD169E030297AD0902978D1012088F898
:102B60000300902088F80400C8F81460C8F81860C2
:102B7000C8F81C60C8F8206000F0F0FB504600F078
:102B8000B9FB80216B48FFF7FAFAA8F80E60C8F885
:102B9000106002F0A5FF00F069FD58E098F803000E
:102BA000F0B38024FF2221466248FFF7E1FA224673
:102BB00009F102015F48FFF7C9FADFF87CA14FF481
:102BC00040794946504601F074FA5A4FD8F810003F
:102BD00000EB850057F8251000F5104000F0CAFB07
:102BE0006D1CADB2202DF1D34946504601F065FA77
:102BF000B8F80E00204481B2A8F80E10D8F81C00D6
:102C0000B1F5006F2044C8F81C00D8F8100020442B
:102C1000C8F810001BD100F5104000F06BFB00E07D
:102C200015E0A8F80E6012E0404D98F804006D1C05
:102C300090280FD088F804600420387187F883004A
:102C4000FFF748FE97F88310485502F041FF002037
:102C5000BDE8F087194688F8042051F8020F00BA41
:102C6000CA7820F0FF001043C8F814004A6899F8A9
:102C7000091012BA22F0FF020A43C8F81820D8F847
:102C80001C204FF0020982420AD151464FF0FF301A
:102C900003F0AAF9C8F82000D8F8181088420DD01F
:102CA00087F80690FFF716FE97F883104855CEE791
:102CB000032C0AD1384600F01DFBC8E745464FF407
:102CC000C0574FF0553941F60408641CE4B2384649
:102CD00000F010FB4946384600F04CFB4046E969DD
:102CE00000F048FB38684845E2D1D8F80000E969AF
:102CF0008842DDD1EE61EE8180210E48FFF73FFA78
:102D0000EE7002F0E5FE00F0A3FC142003F07EF963
:102D1000BFF34F8F09480168094A01F4E06111438C
:102D20000160BFF34F8F00BFFDE700006A05002080
:102D300080000020E8020020005800400CED00E078
:102D40000400FA0570B50F4C0026268060800E48FE
:102D5000A060207C40F0010020744FF08045AE84DC
:102D6000286840F00100286019B1208861888842F5
:102D7000FBD300F02DF9286820F0010028602674AC
:102D800070BD0000740E0020D61800202DE9FC5FF5
:102D9000002426462546A046DFF8E49100F0C2FD57
:102DA00000287DD0774F3988AA2901D076A0DFE0AE
:102DB000DFF8ECA19AF80000F0B340F2234171482B
:102DC000FFF776FD834640F6DA017648FFF7D7F93C
:102DD000B7F8461859457DD14FF4846107EB44009C
:102DE000641CC088A4B2C0F30B0080448C42F5D3AD
:102DF0007888C0B380024FF44872B0FBF2F084B21E
:102E00006948B0FBF4F0804506D94443B4FBF8F0C0
:102E100084B2792C00D27924DFF8888100208B4697
:102E200007EB4001C988C1F30B0239F8101001F01B
:102E30000F03C1F3061C00E016E003EBCC03C90A44
:102E40004FF0670C11FB0CF108EB410101EB430162
:102E5000401C80B28A815845E2D3544900204FF487
:102E6000E67C4B8815E005E09AF80010491C8AF8CA
:102E700000107FE07924C3E707EB4002D288C2F359
:102E80000B08E04507D812050FD0761CB6B2401CDF
:102E900080B28342F0D80120454F4FF0000800E097
:102EA0006CE0B34204D1F87504E06D1CADB2EEE7FE
:102EB00087F81780AB4201D10222FA753D4D0646D4
:102EC0008946A8706020A5F80A80CDE900808B7A39
:102ED000012200E04BE01146002002F0BBF8C820C0
:102EE00003F0ACF84FF480406881182221467A2024
:102EF00002F080F8C82003F0A1F801232E70A5F895
:102F00000A801A461946132002F0D2F899F80A00EE
:102F1000B82100EB400001EB800003F08FF8F87D52
:102F200028B9B87E18B1387F08B100F045FA1022F0
:102F300000212F2002F05EF800F012FB9AF8030047
:102F40005146401CC0B28AF80300782812D181F89B
:102F500003800A794FF400401AB18AF804801649B8
:102F600003E015498AF804601039086002E013A0F4
:102F700002F0BEFDBDE8FC5FFFF7A6BCBDE8FC9F0C
:102F8000246200082C060020686561646572206573
:102F900072726F72203A20307825780A00000000A3
:102FA00002000020FC0F0020E00C301F980F0020D2
:102FB000F0050020C6290020283C024063726320EF
:102FC0006572726F72203A20307825780A0000000E
:102FD00003480168034A928A114301607047000068
:102FE00014340240980F0020194A10B500211160D6
:102FF000174A1432118017490A7C42F001020A7400
:1030000015498A6D22F001028A65CA6E22F001021A
:10301000CA66124A8A670867A2F582724A66C8655C
:10302000886D40F001008865C86E40F00100C866F8
:10303000074C4915103C204602F07BFBA1152046A9
:1030400002F077FB216841F00101216010BD000012
:1030500010040040740E002000000240BA26002038
:1030600006480168C90708D0044914390968C90726
:1030700003D00121016001F0BFBD7047140401407D
:1030800070B5194C2068194D400407D528684004D4
:1030900004D54FF48040206001F0AEFD20680004AC
:1030A00007D52868000404D54FF40040206001F0E3
:1030B000A3FD2068800415D52868800412D50C482B
:1030C000816821F0010181600A48018821F04001F6
:1030D0000180401400F090F807488088BDE87040F7
:1030E00001F08EBC70BD00001404014000040140DA
:1030F00000000240003C0140980F00200648016893
:10310000890708D5044914390968890703D50221BC
:10311000016001F071BD7047140401400648016868
:10312000490708D5044914390968490703D504211A
:10313000016001F061BD7047140401400648016858
:10314000090708D5044914390968090703D5082176
:10315000016001F051BD7047140401400648016848
:10316000C90608D5044914390968C90603D51021D0
:10317000016001F041BD70471404014030B51C4DA1
:1031800028681C4C800606D52068800603D52020C0
:10319000286001F031FD2868400606D52068400609
:1031A00003D54020286001F027FD2868000606D5D9
:1031B0002068000603D58020286001F01DFD2868E6
:1031C000C00507D52068C00504D54FF4807028607D
:1031D00001F012FD2868800509D52068800506D514
:1031E0004FF400702860BDE8304001F005BD30BDEF
:1031F00014040140000401400149086070470000C8
:103200001404014006490968014206D004491439F2
:103210000968014201D0012070470020704700007A
:1032200014040140034B002903D199180A68824312
:103230000A6070470004014010B504460179006837
:1032400000F02EF86179206800F00EF82279A1795B
:103250002068BDE81040FFF7E5BF00210160017163
:103260000C2242718171704730B50C4B0B4D083305
:103270001A6882431A601A1D146884431460102966
:1032800004D029440A6802430A6030BD196801432A
:10329000196011680143116030BD00000004014055
:1032A000064A10B5136883431360131D1C688443DA
:1032B0001C6011440A6802430A6010BD000401400A
:1032C0000249CA680243CA607047000000200240F9
:1032D00000B5034600F02EF802E000F02BF85B1E6C
:1032E000012803D0002B00D1072000BD002BF4D112
:1032F000FAE7000070B505463420FFF7E1FF4FF410
:1033000030263046FFF7E4FF042810D1084C20692E
:1033100040F0020020616561206940F040002061BA
:103320003046FFF7D5FF216921F00201216170BD10
:103330000020024008490420CA68D20701D00120B9
:103340007047CA68520701D502207047C968C9068C
:10335000FBD50320704700000020024003480249CB
:1033600041600349416070472301674500200240E6
:10337000AB89EFCDF0B505460E46800701D006209B
:10338000F0BD3420FFF79CFF4FF400573846FFF79D
:103390009FFF0428F4D1074C206940F00100206110
:1033A0002E603846FFF794FF216921F00101216169
:1033B000F0BD00000020024009480168094BD88890
:1033C00001400948428C0A404284084909691A8927
:1033D0001140828C0A408284816A491C8162704754
:1033E00010380240980F0020F005002000400240F5
:1033F00070B500F031F8174D044602280ED04FF09A
:10340000020116D128896A8800EB01039A4208D983
:10341000501A80B2688000F015F918E04FF00401EE
:10342000EFE7688000F00EF90120A875288B401C9A
:103430000CE0012C0BD168880144E888814200D25D
:1034400088B2688000F0FEF80020A8752883204626
:1034500070BD0000F005002070B5334D688C334E10
:10346000F1880840A8816889E881A88C31890840E2
:103470006882288AA882E87D002138B1012802D01C
:103480000024204670BD02242983FAE7A889EA892E
:103490001040EA89904205D1688AAA8A1040AA8A17
:1034A00090422AD0A87D012825D1E87E012822D18A
:1034B000288BFA281FD3298395F82100D8B9002139
:1034C0000122EB8902FA01F0034206D0AB890342E4
:1034D00003D16B8983436B816B89AB8A034206D02E
:1034E0006B8A034203D12B8A83432B82288A491C8F
:1034F000C9B21029E5D30224C3E7688908B9288A2C
:1035000008B10124BDE70224642002F097FD1F21C9
:103510000022602001F06EFD642002F08FFDF08833
:10352000688130892882ACE7F0050020980F0020E0
:1035300000B587B0802001F0B5F8684600F0E6F9E4
:103540001020009000200390022001900920059097
:103550006946024800F09BF907B000BD0034024004
:1035600070B5354C6078012505285ED2DFE800F0A3
:10357000030E283E5300E07D022856D0607F401C99
:103580006077607F88B36570A5764EE0E07D60BBB4
:10359000A06A032849D9FFF72BFF0221022802D095
:1035A000012804D041E0A07D012803D03DE0A07FA8
:1035B000032801D3617038E0A07F401CA07734E07D
:1035C000642002F03BFD1D4800250178032902D24A
:1035D00000F0D0F808E005700320607044F2F73086
:1035E00060844FF40040A084A5621EE0E07D10B925
:1035F000A06A032802D8E07D012801D1FFF7F8FE78
:10360000E07FA12803D3E576042060700DE0E07F21
:10361000401CE07709E0E07D10B9A06A032802D8D9
:10362000E07D012801D1FFF7E3FE0548C1886184F0
:103630000089A08470BD0000F0050020A4000020D7
:10364000980F00200146014802F069B8003401409B
:103650000449012008700448016841F0010101603B
:1036600070470000F00500200010004002490020D3
:103670000870024908607047F00500200010004003
:103680001FB50446102001F01DF8684602F018F836
:103690003F20641EADF80000ADF8044000200C4C43
:1036A000ADF80600ADF802006946204601F0AEFF15
:1036B0000121204602F041F80121204602F041F8A4
:1036C000204601F06FFF204602F03EF81FBD0000CB
:1036D000001000407FB50D462349B1FBF0F04FF4D8
:1036E0007A71B0FBF1F44FF4005000F0FDFFFFF7EA
:1036F0001FFF684601F0E4FF641E40F2E730ADF8BA
:103700000040ADF804000024184EADF80640ADF8B6
:1037100002406946304601F079FF154AB01511465E
:10372000908170201080D481082050810220108167
:103730000420908001205080D580304602F050F85F
:10374000304601F02FFF09481030016821F00101D7
:103750000160304601F0FDFF304602F097F8044862
:103760002C3845807FBD00000020A10700340140B7
:103770001C06002070B5174D04462978880709D02B
:1037800001F00302012A08D0022A0BD0C8438007A7
:103790000FD013E001F0F0FC0DE0002248F60161CB
:1037A0004E2003E048F240410022462001F022FC76
:1037B00001E001F076FC052002F040FC2878401C76
:1037C000C0B22870042804D1002028702078401C42
:1037D000207070BDAC00002010B514074FEA427293
:1037E0004FEAD2624FF00F0303FA02F301FA02F13B
:1037F00004D5426A9A431143416210BD026A9A435A
:103800001143016210BD10B5C36A520003249440F5
:10381000A34391401943C16210BD0000084A20F043
:10382000030310B51A4453688007C00E3F24844038
:10383000A3435360536881400B43536010BD0000A5
:1038400000000140006980B270470069084000D064
:103850000120704770B50568530003269E4001F0B3
:103860000304B5439C402C430460012905D0112971
:1038700003D0022901D0122908D1436801249440C1
:10388000C1F30011A34391401943416070BD70B56D
:103890000C46064600251DE00120A840014218D034
:1038A0002A4630466169FFF797FF2A46304661682D
:1038B000FFF7D0FF2A463046A16800F014F82A46E8
:1038C0003046E16800F019F82A4630462169FFF7D2
:1038D0009AFF6D1C216831FA05F0DDD170BD81625F
:1038E00070478161704710B5C3685200032494404B
:1038F000A34391401943C16010BD10B583680124F2
:103900009440A34391401943816010BD4FF6FF716D
:1039100001600021C16041600F228160C0E9041292
:103920007047000002480078002800D0012070474E
:10393000A600002070B506460024A7E014B955A0E3
:1039400002F0D6F880251CB9294657A002F0D0F81D
:1039500000222946412001F04DFB642002F06EFB5D
:1039600000251CB9294654A002F0C2F800222946BD
:10397000422001F03FFB642002F060FB04251CB9EB
:10398000294651A002F0B4F800222946472001F050
:1039900031FB642002F052FB4AF634251CB929465B
:1039A0004DA002F0A5F800222946482001F022FB94
:1039B000642002F043FB4FF404451CB929464AA099
:1039C00002F096F800222946492001F013FB6420FA
:1039D00002F034FB19251CB9294647A002F088F8EB
:1039E000002229464A2001F005FB642002F026FB54
:1039F00000251CB9294644A002F07AF80022294685
:103A00004B2001F0F7FA642002F018FB42F208059F
:103A10001CB9294640A002F06BF8002229464C2030
:103A200001F0E8FA642002F009FB49F601651CB9CF
:103A300029463DA002F05CF8002229464E2001F004
:103A4000D9FA642002F0FAFA4FF4C0451CB92946AD
:103A500039A002F04DF8002229464F2001F0CAFAA1
:103A6000642002F0EBFA384800F056F9FF250022F6
:103A70002946402001F0BEFA1CB9294633A002F0C5
:103A800037F8642002F0DAFA641CE4B2B442FFF4BE
:103A900055AF70BD0A0A72656769737465722063F9
:103AA0006F6E6669670A00007265675F34313A308D
:103AB0007825780A000000007265675F34323A307A
:103AC0007825780A000000007265675F34373A3065
:103AD0007825780A000000007265675F34383A3054
:103AE0007825780A000000007265675F34393A3043
:103AF0007825780A000000007265675F34413A302B
:103B00007825780A000000007265675F34423A3019
:103B10007825780A000000007265675F34633A30E8
:103B20007825780A000000007265675F34653A30D6
:103B30007825780A000000007265675F34463A30E5
:103B40007825780A00000000AE0000207265675FEB
:103B500034303A307825780A000000002DE9F05F13
:103B60000024642002F052FA641CA4B2052CF8D39D
:103B7000554D00224FF64003A87A401E81B21046F0
:103B800002F03CFB002445F6C3274FF4804601F0C9
:103B9000F3FA642002F052FA01F0F4FA642002F021
:103BA0004DFA022C05D1002233461146104602F090
:103BB0002FFB39460022682001F01CFA642002F035
:103BC0003DFA641CA4B2032CE1D3DFF800A1DFF8B6
:103BD00000B100244FF6FF7844F2F73900231A466B
:103BE0001946184602F014FBA97A012001F0DEF90B
:103BF000A87A401DC0EB001000EB800108EA8100AC
:103C000002F01CFA5046FFF71DFE07465846FFF724
:103C100019FE17EA090F0CD0032C17D22D48468144
:103C200001F0B0FA4FF4FA7002F008FA022C07D053
:103C30000CE000231A461946184602F0E9FA09E09A
:103C400000231A461946184602F0E2FA641CA4B290
:103C5000032CC3D300244AF2C95529460022682008
:103C600001F0C8F9642002F0E9F9641CA4B2032C45
:103C7000F3D30320FFF75EFE002448F642463546A4
:103C80001CB9314614A001F033FF0022294646201A
:103C900001F0B0F9642002F0D1F93F251CB92946A2
:103CA00011A001F025FF00222946602001F0A2F9B1
:103CB000642002F0C3F9641CA4B2032CDFD3BDE876
:103CC000F05F0DA001F014BF980F002000380240F3
:103CD00000400240C62900207265675F34363A30E2
:103CE0007825780A000000007265675F36303A3048
:103CF0007825780A000000006261636B6C69676870
:103D0000742064726976657220696320696E6974D3
:103D100020646F6E650A00002DE9F84FDFF870A08F
:103D200081460021194ADFF86CC09AF800709AF8B1
:103D300001801AE0002014E032F8023B39F811400B
:103D400003F00F05C3F3061605EBC605DB0A67266D
:103D500013FB06F30CEB430303EB4503401C9C8170
:103D6000C0B28742E8D8491CC9B28845E2D8BAF83F
:103D70000C0000909AF80A3008220121502001F02E
:103D80004FF9BDE8F84F642002F058B924620008EA
:103D9000980F0020FC0F002010B5194C204600F0B1
:103DA00090F9B0F5806F06D01649C20509D508888C
:103DB00020F480700AE02046BDE81040124900F06F
:103DC0004EB9820504D5088820F40070088010BD23
:103DD000020503D5088820F40060F7E7C20403D584
:103DE000088820F48050F1E7420403D5088820F4C5
:103DF0008040EBE70004EAD5088820F40040E5E7BE
:103E00000058004014580040000400102DE9F0470D
:103E1000DFF840A1504600F054F9C1033ED4DFF86A
:103E200038814C4A4D4F4E4B01251032DFF834910A
:103E30007C1FA0EB08014FF0000CA3F580764045F5
:103E400052D013DCB0F1021F26D003DC48B1102899
:103E50001ED179E04038B0F500306FD04249C842F9
:103E600016D15046BDE8F04700F032B9DFF8FC80CB
:103E7000A1EB080041450FD004DC022910D0042931
:103E800006D131E03E2859D07E38B0F5802F07D0DA
:103E9000BDE8F04700F0B2B9A4F80AC0BDE8F08769
:103EA000A4F80CC0307820280FD1707801280CD1EC
:103EB000B078012802D0022804D006E0F07820284B
:103EC00021D002E0F07820280CD0484650F8061F98
:103ED000196041685960B9F80E001881187810808F
:103EE000A581DBE73878FAE73078202811D170789F
:103EF00001280ED1B078012802D0022806D008E0AF
:103F0000F078202805D1A0781080C7E7F078202825
:103F100010D0484650F8061F196041685960B9F83A
:103F20000E001881207B00F00F00195C1180401CEE
:103F3000A081B3E7A089395CF8E7FFE7A07A118890
:103F40003154401C6081A9E7504600F0C1F825813A
:103F5000A4E7000000580040800006008500002013
:103F6000E8010020646A00083C00FCFF82FF7B003F
:103F7000028822F480620A4302807047028922F498
:103F800000420A4302817047028822F00A020A4373
:103F90000280704770B586B0044616460D466846E6
:103FA00000F0B4FBA088029920F03F022648B1FB44
:103FB000F0F080B2202800D920200243A28022887D
:103FC00022F001022280226A22F03F031F4A95421A
:103FD00012D86A00B1FBF2F189B2042900D204219F
:103FE000401C00F03F0018432062A183208840F06D
:103FF0000100208006B070BDB6F5804F05D005EBFE
:104000004502B1FBF2F18AB208E005EBC50202EB12
:104010000512B1FBF2F189B241F48042110501D1E0
:1040200042F001020A4E42F400414FF47A72B54266
:1040300003D84FF49675684302E0C0EB0010C0004F
:10404000B0FBF2F0CCE7000040420F00A086010078
:10405000801A0600818941F0010181817047C943BE
:104060008182704770B50C46CA8805460968FFF71B
:1040700091FFA1882846FFF787FF61892846FFF74F
:1040800077FFA1892846FFF779FF21892846BDE8F7
:10409000704000F022B841F2883101600021818037
:1040A0004BF6FF72C280018141814FF480418181D2
:1040B000704782888A438280704782880A43828060
:1040C0007047818A008B41EA004121F07F407047B0
:1040D000018841F001010180704702896FF30902F4
:1040E0000A4302817047828901F0FE0122F0FE023C
:1040F00011438181704700000449884202D14FF486
:10410000001001E04FF4800000F0E4BA00540040D9
:1041100030B58BB04FF4807000F0C4FA4FF48000DB
:1041200000F0D0FA6846FFF7F1FB4FF440600090D2
:10413000122001900720059000240120CDE90204FF
:1041400069461748FFF7A3FB164D2846FFF7D4FF33
:1041500006A8FFF7A0FF29144C20ADF82000081195
:10416000ADF82200ADF81C400F48ADF81E10ADF8B8
:104170002410069046212846FFF7B5FF2846FFF792
:1041800069FF06A92846FFF76DFF4FF4E061284656
:10419000FFF793FF2846FFF79BFF0BB030BD0000F1
:1041A0000038024000580040A086010030B50021D0
:1041B000034608464FF6FF74012505FA01F204EAAA
:1041C00040001A4201D040F00100491CC9B2102938
:1041D000F3D330BD0249084302490860704700002C
:1041E0000000FA050CED00E0024A114001430248CC
:1041F0000160704780FFFF1F08ED00E010B54FF42D
:104200008004204600F066FA204600F053FA20466B
:1042100000F060FAFFF77CFF202001F086FCBDE88B
:104220001040212001F081BC70B5084E084C0025DB
:10423000208938B1357061890648FEF70FF8FEF71E
:1042400067FC2581E0780028F2D170BD680300206A
:1042500080000020E800002038B5174C00200090B6
:10426000144D206820F080002060206840F040005D
:10427000206069461148A8470098C0B2052814D8A4
:1042800069460F48A84700984FF47F42010E02EAA2
:104290001022114300F47F400A4A41EA00210091B4
:1042A000106800F07F4008431060206840F08000F4
:1042B000206038BDA502FF1F0020024020F0FF1F34
:1042C00030F2FF1F0418004010B54FF48034204630
:1042D000FEF798FF00280AD005490120087005A0C4
:1042E00001F006FC2046BDE81040FEF785BF10BD7A
:1042F000AA000020700A00001CB54FF0805000F0AA
:10430000E1F96846FEF7A9FF4FF480342046FEF736
:1043100073FF00208DF8040010208DF805000120A7
:104320008DF8060000946846FEF786FFE02000F056
:1043300009F80348016841F0100101601CBD00004C
:1043400000700040034A116821F438710143116084
:1043500070470000007000402DE9FF4F074682B013
:104360002A484FF6FF71DDF83C8091460025818296
:10437000284A2749D160284C4FF0100B04F582766B
:10438000824616E037F81500010A8AF8101017F86F
:1043900015108AF81010CDE9008B34F8023C37F87C
:1043A000150032462146FEF705F96D1C2034EDB2AA
:1043B000203603988542E5D357460025DA4614E0B7
:1043C00039F81500000A387419F81500387439F8EE
:1043D0001500CDE9008A34F8023C32462146FEF74A
:1043E000E9F86D1C2034EDB2203605988542E7D3FC
:1043F000B88ACDE9008A34F8023C32462146FEF7FD
:10440000D9F8A4F81E8006B0BDE8F08F0030024055
:1044100000340240740E0020D82500202DE9F0471A
:10442000DFF864900E464FF6FF711D469046074632
:104430000024A9F8141045F2555018807200981CF9
:104440003946FDF783FE701C80B24B4608E037F812
:104450001410090A197417F814101974641CA4B202
:10446000B442F4D3002108E035F81020140A1C747B
:104470001A74401C491C80B289B24145F4D3998A10
:1044800025F81010BDE8F0870030024070B5314CBF
:1044900000206021A073A1810B21E17349F6E7514F
:1044A000A18244F2F731E1804FF4004121810C21D7
:1044B000A1722949216129492162294905466722BA
:1044C000424304EB800301EB42025A63401CE27B4F
:1044D000C0B28242F3D8182060702C2020704FF4B4
:1044E00084616180081DA0801EA001F001FB21787D
:1044F00021A001F0FDFA617824A001F0F9FA607FB3
:1045000008B127A100E02AA12DA001F0F1FAE17B7A
:104510002FA001F0EDFAA27AA18933A001F0E8FA08
:1045200047F2305060834FF4967020833A4840F24F
:10453000F521C1800581E18841812289028241847F
:104540008284856280F821500221C17501210177A2
:10455000457070BD980F00201A00002024620008EA
:10456000FC0F002070726F6A656374207A6F6E654D
:10457000733A25640A00000070726F6A65637420E4
:1045800077696474683A25640A00000070726F6A83
:10459000656374206865696768743A25640A000079
:1045A00068696768207370656564206D6F64650075
:1045B0006C6F77207370656564206D6F64650000B3
:1045C000737062206D6F64653A25730A0000000005
:1045D00070726F6A656374206469206E756D6265C0
:1045E00072733A2564200A0070726F6A65637420E2
:1045F000646920636173636164653A2564202C20DB
:104600006963206E756D62657220706572206469E1
:10461000703A25640A000000F0050020114810B52A
:10462000017800291DD0002101700FA001F060FA6F
:104630000DA001F05DFA0CA001F05AFA11A001F0F2
:1046400057FA322001F0E2FCBFF34F8F13480168A4
:10465000134A01F4E06111430160BFF34F8F00BFC3
:10466000FDE710BDAA0000206F63637572205643FA
:1046700043206C657373207468616E203256390A6A
:1046800000000000726561647920746F20726573A8
:10469000746172742062636F6E0A00000CED00E0BA
:1046A0000400FA0502494A6902434A617047000062
:1046B000001002400249CA698243CA617047000083
:1046C000001002400249CA690243CA6170470000F3
:1046D0000010024003490A6902430A610A698243E1
:1046E0000A6170470010024002498A6902438A61E8
:1046F00070470000001002400349CA680243CA60C4
:10470000CA688243CA6070470010024030B5284B27
:104710005968284A11405A680C0102F4803201D4C9
:10472000022401E06FF4F77404EB91411AB15A6866
:10473000920305D502E01A6CD20701D01E4A00E0B0
:104740001E4A51435A681D4C12F00C0203D0042A31
:1047500001D0082A01D0046000E001605A68184CBA
:10476000C2F30312A55C0268EA4042605D68C5F3CB
:104770000225655D22FA05F585605D68C5F3C225F1
:10478000645D22FA04F4C460DC6A0D4D04F00F0489
:1047900010352C5DB2FBF4F24261DA6A05F11003C8
:1047A000C2F3031233F81220B1FBF2F1016130BD04
:1047B0000010024000003C0800093D0000127A0091
:1047C000746E0008028822F03802028002880A43D0
:1047D00002807047028822F00102028002880A43A8
:1047E00002807047028822F00202028002880A4397
:1047F00002807047028822F44442028002880A4301
:1048000002807047028822F40062028002880A4314
:1048100002807047028822F08002028002880A43E8
:104820000280704782880A43828070470649884226
:1048300001D1801404E00549884203D14FF40020DF
:10484000FFF75ABF7047000000300140003C0140B4
:1048500010B50B4604460988FFF7CCFF598820465F
:1048600000F034F899882046FFF7CCFF19892046DC
:10487000FFF7B0FFD9882046FFF7B4FF59892046DB
:1048800000F017F899892046FFF79CFFD989204648
:10489000FFF7C0FF188A208210BD002101804180EF
:1048A0008180C180018141818181C1810721018293
:1048B0007047028822F40072028002880A43028054
:1048C0007047018821F0400101807047028822F082
:1048D0000402028002880A430280704710B54FF438
:1048E000A060FFF777FC0120FFF7FEFE00211B20F0
:1048F00001F028F900211C2001F024F905212720CE
:1049000001F020F905210B2001F01CF90A210D20EE
:1049100001F018F90A210F2001F014F909212020D3
:1049200001F010F90A21212001F00CF909211D20C4
:1049300001F008F90A212F2001F004F90F210120CC
:1049400001F000F90A21302001F0FCF80A212420AE
:1049500001F0F8F80121062001F0F4F80121072008
:1049600001F0F0F80121082001F0ECF80121092004
:1049700001F0E8F801210A2001F0E4F801211620F5
:1049800001F0E0F8272001F0C3F8062001F0C0F89C
:10499000072001F0BDF8082001F0BAF8092001F065
:1049A000B7F80A2001F0B4F8162001F0B1F80B2096
:1049B00001F0AEF80D2001F0ABF80F2001F0A8F8DF
:1049C0001B2001F0A5F81C2001F0A2F81D2001F029
:1049D0009FF82F2001F09CF8012001F099F8202089
:1049E00001F096F8212001F093F8302001F090F8C2
:1049F000242001F08DF8BDE81040802000F014BDA7
:104A00001549CA6842F40022CA60CA6822F400222A
:104A1000CA608A6942F400228A61104900230B802F
:104A20000A1D1380138843F0010313800A8842F49F
:104A300020620A800A8842F040020A8008498A6897
:104A400022F001028A60074A4A61C860886840F023
:104A5000010088607047000000100240003C0140E7
:104A6000000002402C06002070B5324D90B0284660
:104A7000FFF7DCFE4FF40020FFF736FE0120FFF7C2
:104A800011FE0BA8FFF709FF0024E814ADF8300071
:104A9000ADF834408010ADF836000120ADF82C4060
:104AA000ADF83840ADF83C00ADF82E40ADF83240DE
:104AB000ADF83A400BA92846FFF7CAFE1E4E304615
:104AC000FDF7CAFF6846FEF715F81A4869460C302C
:104AD00000901A48CDE9010440F22440CDE90304D6
:104AE00080200590400006908000CDE907044FF437
:104AF0004050CDE909043046FDF753FF0E4908390F
:104B00004C60886840F002008860886940F00B00C3
:104B1000886101212846FFF785FE0C213046FDF70C
:104B20002EFF3046FDF726FF2846FFF7CAFE10B0DD
:104B300070BD0000003C0140080002402C0600202F
:104B400010B586B08020FFF7ADFD6846FEF7DEFEAB
:104B500001200021274C01900391009069462046D6
:104B6000FEF795FE0221009169462046FEF78FFE72
:104B70000421009169462046FEF789FE0821009134
:104B800069462046FEF783FE2020009069462046B5
:104B9000FEF77DFE4020009069462046FEF777FE36
:104BA0008020009069462046FEF771FEA015009017
:104BB00069462046FEF76BFE2015009069462046A8
:104BC000FEF765FEE014009069462046FEF75FFEA2
:104BD000A014009069462046FEF759FE4FF40040AD
:104BE000009069462046FEF752FEFEF7F1F906B046
:104BF00010BD00000034024030B50D4801780D4A68
:104C0000002341B114880C4908888D680544401C74
:104C100008802C700AE001210170064814380360F6
:104C200004482438016841F001010160138030BD5F
:104C3000AB00002024080040880E002070B54FF41F
:104C400080758AB02846FFF72DFDA800FFF72AFDE2
:104C50000120FFF749FD0420FFF734FD0820FFF78E
:104C600031FD6846FEF752FE00240121CDE9021411
:104C7000684E0091019469463046FEF708FE012116
:104C80000020FEF7CBFD0220009069463046FEF77B
:104C9000FEFD05210120FEF7C1FD042000906946BC
:104CA0003046FEF7F4FD09210220FEF7B7FD08208B
:104CB000009069463046FEF7EAFD0D210320FEF71D
:104CC000ADFD1020009069463046FEF7E0FD112151
:104CD0000420FEF7A3FD2020009069463046FEF731
:104CE000D6FD15210520FEF799FD4020009069466C
:104CF0003046FEF7CCFD19210620FEF78FFD8020FF
:104D0000009069463046FEF7C2FD1D210720FEF7E0
:104D100085FD694630460095FEF7B9FD2121082042
:104D2000FEF77CFD6800009069463046FEF7AFFD57
:104D300025210920FEF772FDA80100906946304642
:104D4000FEF7A5FD39210E20FEF768FDE801009071
:104D500069463148FEF79BFD3F210F20FEF75EFDBF
:104D60002E49C888098908432D490A6882430A6088
:104D70002B4908310A6802430A60091D0A6810437A
:104D8000086006A800F09CFC9F20ADF81C000325DD
:104D9000244EADF81850ADF81E40ADF81A4006A9E3
:104DA000304600F033FC304600F0FCFB294630462C
:104DB00000F084FC1B491031086820F001000860F5
:104DC0000121304600F0B9FC06A800F079FC40F65D
:104DD0009F70ADF81C00ADF81840ADF81E40ADF85E
:104DE0001A40114C0F2506A9204600F00FFC204662
:104DF00000F0D8FB2946204600F060FC0A4910313B
:104E0000086820F0010008600121204600F095FCB0
:104E10000AB070BD0038024000400240980F0020E8
:104E20000004014000080040000C004010B5FFF7EE
:104E300087FEBDE81040FFF701BF0000054801688C
:104E400021F0010101600448016821F001010160C5
:104E50007047000000080040000C00402DE9F041C0
:104E600094B00120FFF72EFC0220FFF72BFC01205D
:104E7000FFF718FC0BA800F023FC05270024ADF871
:104E80003070ADF82C40BD070626ADF83240ADF8C5
:104E90002E400BA9284600F0B9FB284600F082FB03
:104EA0003146284600F00AFC286920F001002861FC
:104EB0000121284600F041FC0BA800F001FC09206C
:104EC000ADF83000344EADF82C400725ADF8324037
:104ED000ADF82E400BA9304600F098FB304600F0AC
:104EE00061FB2946304600F0E9FB6020ADF83C004C
:104EF0000120ADF83E00ADF84440ADF842700FA976
:104F0000304600F02BFC7115304600F012FCB7154E
:104F10003946304600F00DFC1F48103004601F4E2B
:104F20003046FDF799FDDFF87480A8F1140840467B
:104F3000FDF792FD6846FDF7DDFD1A48184DCDE9F5
:104F400000501020CDE902048020CDE904400697EE
:104F5000C000CDE907044FF44050CDE9090469468B
:104F60003046FDF71EFD10486946CDE90050404629
:104F7000FDF717FD1D213046FDF701FD20214046BC
:104F8000FDF7FDFC05486C38816D41F0020181653B
:104F900014B0BDE8F0810000000400406C00024045
:104FA00014340240BA260020B625002038B500226D
:104FB000ADF800200C4A47F2B04340EA01241278D1
:104FC00043EA0215094A137C002BFCD10848807B78
:104FD00000B1012001F0E4F86B460022214628468A
:104FE00000F092F838BD0000C6290020740E0020A1
:104FF000980F0020F7B5094B0446002542F4E4461B
:10500000187C0028FCD1012001F0CAF801AB22462F
:105010002946304600F078F8FEBD0000740E0020EE
:10502000F0B41B0205460A48A3F580730B43120235
:105030000078A2F58072049C4FF4E64699B22A43A8
:1050400046EA00102346F0BC92B200F0A1B800007E
:10505000C6290020F0B414460646DDE904250948B7
:105060000170807840EA01104FF4E24141EA4601C4
:1050700008431902A1F5807121432B46F0BC89B287
:1050800000F086B8C629002010B5FFF7CFFEFFF765
:10509000E5FE4020FFF706FBBDE81040012001F0CF
:1050A0007FB8002245F6C3217820FFF7A3BF000098
:1050B000F8B504460020ADF8000010484FF4EA456A
:1050C000007845EA00161802A0F58070084385B202
:1050D0001002A0F580702043094B84B2187C002890
:1050E000FCD10848807B00B1012001F059F86B46E3
:1050F00022462946304600F007F8F8BDC6290020B0
:10510000740E0020980F002030B5154687B0024677
:1051100000201C46049005900690ADF80C00ADF8F8
:1051200010200846FFF742F8ADF812002846FFF7B6
:105130003DF8ADF814000E480189ADF8161040890D
:10514000FFF734F8ADF818000A4805210123808ADA
:105150000090224604A8FFF7FFF88120ADF80C006C
:105160000121BDF80C00FDF73FFF07B030BD000086
:10517000C6290020980F002000224AF2C951782049
:10518000FFF738BF00224AF2C9517C20FFF732BF37
:105190002DE9FE4300240094ADF800001D4616469C
:1051A000019402940846FFF701F8ADF8020030467A
:1051B000FEF7FCFFADF8040016480189ADF80610B3
:1051C0004089691E084380B2FEF7F0FFADF8080081
:1051D000280170304FF005091FFA80F80E4E0F4F6E
:1051E0000BE0672014FB00F006EB40032A4649461B
:1051F0006846FFF713F9641CE4B2F87BA042F0D8CC
:105200004046FDF7B1F801214046FDF79BFDBDE8A2
:10521000FE830000C6290020FC0F0020980F00200C
:105220000648016811B10168491E016081680029C2
:1052300002D04168491C41607047000074000020A2
:1052400070B586B00120FFF74FFA4FF48070FFF77A
:1052500029FA6846FEF75AFB01244FF40050022554
:105260000594CDE900050D4E69463046FEF70FFB6B
:1052700020030594CDE9000569463046FEF707FB9B
:10528000E003009000200190694605943046FEF747
:10529000FEFA06B0BDE87040FFF7E6BB00380240FA
:1052A0003EB5002000908DF80400324C029020683A
:1052B00040F0010020604FF4A0612068C0F340007E
:1052C0008DF804000298401C02909DF8040010B96B
:1052D00002988842F1D12068C0F340008DF80400A4
:1052E0009DF80400F0B32448016821F00701016033
:1052F00022490968016841F003010160606860604B
:10530000606840F400506060606840F4A0606060D5
:10531000FEF7A2FF60681A4908406060206C20F028
:1053200001002064606801900098164940F0010077
:105330000090019808430190606000982064206804
:1053400040F08070206020688001FCD5606820F00B
:1053500003006060606840F0020060606068C0F355
:10536000810000E002E00228F8D13EBD074906486E
:1053700008603EBD0010024000200240002004E012
:10538000FFFFC0F700003C0800127A00E000002098
:105390001E4810B5016841F4700101601C480168A5
:1053A00041F00101016041681A4A11404160016801
:1053B000194A11400160016821F4802101604168AF
:1053C000164A114041604FF46051C162016C41F0D6
:1053D0000101016412498160C16941F08051C161DC
:1053E000C16921F08051C1610E48016841F080011E
:1053F0000160016821F010010160FFF751FF0349CE
:105400004FF000608039086010BD000088ED00E0BA
:10541000001002400CC07FF8FFFFF6FEFFFFC0F750
:1054200000009F04002002404FF47A7148434FF07F
:10543000E02100220A6148618A6106200861704704
:1054400070B5104C20681049898A4840231D1860A7
:10545000002519070D610D480288521C0280028840
:105460004688B24204D10A6822F001020A600D6146
:10547000216882681288514019608168891C8160A6
:1054800070BD000010340240980F0020740E002000
:10549000104810B5002101600F48028843889A42E5
:1054A00009D28168028831F81210C26851610188FE
:1054B000491C018010BD094B1A68094CA48A22437B
:1054C0001A60044A103A136823F001031360017450
:1054D00010BD000010040040740E0020143402407F
:1054E000980F00200E4A00B51068C00716D0FFF7CD
:1054F000A5FC106820F0010010600949002014315B
:1055000008800848C18800890143074802688A4327
:1055100002600648017B41F00101017300BD0000FB
:1055200010080040980F002000040140880E002061
:105530000D4800B5016821F0010101600B4A506877
:10554000401E5060506800280DD1FFF777FC0848D6
:10555000C18800890143074803688B430360107BBF
:1055600040F00200107300BD100C0040880E0020B7
:10557000980F0020000401400848016921F0010152
:10558000016107480188491C01800188B1F5FA6F63
:1055900002D34FF4C8610180704700000010004042
:1055A000A8000020016841F08001016070470029D7
:1055B000016802D041F4006101E021F40061016062
:1055C00070470029016802D041F4805101E021F4C4
:1055D0008051016070470029016802D041F40051F8
:1055E00001E021F40051016070470029016802D0F8
:1055F00041F4804101E021F480410160704702687C
:1056000022F070020A4302607047000070B5214D1D
:105610000C460346A84206D06188FFF7F0FFE188F8
:10562000184600F074F8A0889885208818851A4AD2
:105630001A4E934201D0B34201D1207A188601203C
:105640009882AB4203D0617A1846FFF7B0FF4FF063
:105650008045934209D0B34207D0AB4205D01048F1
:10566000834202D00F48834213D1617B184600F079
:105670001BF8AB420DD1A17A1846FFF7A2FFE17AE1
:105680001846FFF7A8FF217BBDE870401846FFF7DA
:10569000ACBF70BD00100040002C01400034014040
:1056A00000040040000800400029016802D041F4D5
:1056B000004101E021F4004101607047018570471D
:1056C0004FF6FF71818000210180C180418001720D
:1056D00041728172C1720173417381737047026AB2
:1056E00001238B409A4302627047026A01238B4078
:1056F0001A4302627047026A04238B409A43026293
:105700007047026A04238B401A43026270470268A2
:1057100022F44072026002680A4302607047C26B62
:105720006FF30F020A43C263704782898A43828102
:10573000704782890A438281704782890A43828145
:105740007047C94301617047016821F001010160A0
:105750007047016841F0010101607047F0B50C46E7
:1057600005460021FFF7BBFF6E68288B278820F0D5
:105770007300074321890022284600F07EF86088E4
:105780004FF000010028284602D0FFF7AEFF01E0ED
:10579000FFF7A5FF1048854202D01048854215D179
:1057A00061890022284600F05FF8A0884FF00001D0
:1057B0000028284602D0FFF7A4FF01E0FFF79BFF77
:1057C00026F44071A089E689084306436E602F8362
:1057D000E0886863F0BD0000002C01400034014007
:1057E000F0B50C4605460821FFF779FF6E68E869B9
:1057F000278880B220F073000743218908222846B9
:1058000000F03BF860884FF008010028284602D0DD
:10581000FFF76BFF01E0FFF762FF1148854202D0FE
:105820001048854217D161890822284600F01CF8EB
:10583000A0884FF008010028284602D0FFF761FF3A
:1058400001E0FFF758FFA18926F4405040EA01101B
:10585000E18940EA01166E60EF61E088E863F0BD1F
:10586000002C01400034014010B5036A0824944024
:10587000A34391401943016210BD10B5036A02248D
:105880009440A34391401943016210BD30F8441F76
:1058900041F400410180704730B587B004460D46A1
:1058A0006846FEF733FF1448844205D013498C4202
:1058B00002D013498C4201D1039A00E0029AA90058
:1058C00002EBC20000EB0210B0FBF1F16423B1FB6C
:1058D000F3F0020110096FF01805684301EB800036
:1058E000322101EB0010B0FBF3F000F00F00104389
:1058F000208107B030BD0000003801400050014059
:1059000000540140C1F3080181807047818941F44E
:105910000051818170470088084000D00120704705
:10592000828A22F440720A438282704770B50C4624
:1059300005460968FFF7B0FFA188284600F053F834
:10594000E188284600F03EF82189284600F010F84A
:105950006189284600F006F8A1892846BDE8704014
:10596000FFF7DEBF828922F00C020A438281704772
:10597000828922F4C0620A43828170470D498842BD
:1059800002D14FF4804011E00B494FF400328842BD
:1059900002D11046FEF79EBE0849884201D110464A
:1059A00004E00749884203D14FF48020FEF7A4BEEB
:1059B00070470000003801400044004000500140A2
:1059C00000540140028A22F440520A430282704786
:1059D0004FF41651016000218180C18001810C22A9
:1059E000428181817047828922F480520A438281F8
:1059F0007047000030B504468BB04FF48070FEF75E
:105A000051FE44F20100FEF76FFE04A8FDF77EFF91
:105A10004FF400700490022005900520099004A91D
:105A20000F48FDF734FF0F4D2846FFF7A7FF6846E4
:105A3000FFF7CEFF0020ADF80400ADF80600ADF88A
:105A40000800ADF80C000820ADF80A000094694683
:105A50002846FFF76BFF2846FFF758FF0BB030BD15
:105A600000340240003801401CB500F019F8012054
:105A7000FEF73AFE36210D20FDF7D0FE4FF4005020
:105A8000009000208DF8040008208DF8050001200A
:105A90008DF806006846FDF7CFFB00F021F81CBD2D
:105AA00000B587B04FF40070FEF7FCFD6846FDF7C7
:105AB0002DFF00200221CDE9010103900803009091
:105AC00069460248FDF7E3FE07B000BD003C024016
:105AD0000248016841F40051016070470804014028
:105AE0000248016821F40051016070470804014038
:105AF0000FB4054B10B503A9044A029800F042F810
:105B000010BC5DF814FB000065600008E400002094
:105B1000002809DB00F01F020121914040098000AC
:105B200000F1E020C0F800117047002809DB00F008
:105B30001F02012191404009800000F1E020C0F8DF
:105B4000001170470907090E002804DB00F1E0206E
:105B500080F80014704700F00F0000F1E02080F89A
:105B6000141D704702E008C8121F08C1002AFAD1AC
:105B700070477047002001E001C1121F002AFBD1CD
:105B8000704700002DE9FF4F8DB00F4605460026F7
:105B900006E025280BD0DDE90F1290476D1C761C1E
:105BA00028780028F5D111B03046BDE8F08F0024E8
:105BB000A246A1460122EC4900E0044315F8013F4A
:105BC000203B02FA03F00842F7D128782A2810D0A7
:105BD0006FF02F022878A0F13001092914D80AEBC0
:105BE0008A0102EB410144F0020400EB010A6D1C42
:105BF000F0E701CF5FEA000A03D544F40054CAF18C
:105C0000000A44F002046D1C28782E2817D115F8DC
:105C1000010F44F004042A280ED06FF02F022878D8
:105C2000A0F1300109290AD809EB890102EB4101F1
:105C300000EB01096D1CF2E757F8049B6D1C2878F6
:105C40006C280FD006DC4C2817D068280DD06A28A5
:105C500014D104E0742810D07A280FD10DE044F458
:105C600000140AE044F4801401E044F4401469781C
:105C7000814202D104F580146D1C6D1C2A786E2AB5
:105C80001FD00CDC632A31D004DC002A8BD0582AC8
:105C900011D1A3E0642A68D0692A0CD165E0732A87
:105CA0002ED004DC6F2A73D0702A04D19BE0752AB1
:105CB0006FD0782A6ED01046DDE90F129047761C1F
:105CC00050E1C4F30250022806D0032809D004286A
:105CD00001CF09D0066045E101CFF117C0E90061AD
:105CE00040E101CF06803DE106703BE117F8040B6F
:105CF0008DF8000000208DF80100EB46012003E044
:105D000057F804BB4FF0FF3061074FF0000102D499
:105D10000DE008F10101884649450FDA8045F8DBBE
:105D20001BF808100029F4D108E008F101018846A9
:105D30008142FADB1BF808100029F6D1DDE90F23B8
:105D4000AAEB08008146214600F036F9304400EB0A
:105D5000080604E0DDE90F121BF8010B9047B8F1CB
:105D60000108F7D221464846F7E00A21C4F302535E
:105D70004FF0000B0891022B04D001CFC117032B69
:105D800009D00AE0FF1D27F00707F7E8020108E045
:105D900032E01FE020E000B2C117042B01D140B275
:105DA000C117031E71F1000307DA4FF0000CD0EBAE
:105DB0000C006CEB01012D2302E0230504D52B23FD
:105DC0008DF82430012303E0E30701D02023F7E717
:105DD000984658E00A2110E010210EE010204FF004
:105DE000000B08900CE010214FF0000B44F004046D
:105DF0004FF00809089103E008214FF0000B0891CB
:105E0000C4F30253022B04D001CF0021032B06D090
:105E100006E0FF1D27F00707F7E8020103E080B264
:105E2000042B00D1C0B24FF0000823072BD5702AF5
:105E300007D0DDF820C08CF0100C5CEA0B0C05D00C
:105E40000EE040238DF82430012308E050EA0103DE
:105E500006D030238DF824308DF825200223984673
:105E6000DDF820C08CF0080C5CEA0B0C0BD150EA7A
:105E7000010301D1630706D530238DF824304FF09C
:105E80000108A9F10109582A04D038A20B9208AAE6
:105E90000A920BE03AA2F9E75B46089AFCF77AF916
:105EA0000B9B9B5C0A9A521E0A92137050EA0102E5
:105EB000F2D10A98ADEB000000F1200B600702D58B
:105EC00024F4803401E04FF00109D94502DDA9EB4B
:105ED0000B0000E0002000EB0B0141440890AAEB0E
:105EE000010AE00306D4DDE90F232146504600F005
:105EF00063F806444FF0000908E009A911F8090009
:105F0000DDE90F12904709F10109761CC145F4DB68
:105F1000E0030CD5DDE90F232146504600F04CF894
:105F2000064404E0DDE90F1230209047761C089902
:105F3000481E08900029F5DC08E00A980A990078C4
:105F4000491C0A91DDE90F129047761CBBF1000154
:105F5000ABF1010BF1DC21465046DDE90F2300F0E7
:105F600019F806446D1C1BE6092801003031323354
:105F70003435363738396162636465660000000085
:105F8000303132333435363738394142434445466F
:105F9000000000002DE9F041044600251E4617468A
:105FA000880404D405E039462020B0476D1C641EE7
:105FB000F9D52846BDE8F0812DE9F04104460025D9
:105FC0001E469046C80301D5302700E020278804EC
:105FD00004D505E041463846B0476D1C641EF9D52E
:105FE0002846BDE8F081000030B50023064C07E0EC
:105FF000CD5C5B1C85EA106554F8255085EA0020CD
:106000009342F5DB30BD0000746A0008822800D995
:1060100082204FF0E02104230B614FF4FA32504309
:10602000486100228A61052008610869000CFCD0E3
:106030000B614FF4FA3048618A6170474FF0E021FC
:1060400004220A61C001486100238B6105200861B8
:10605000086910F4803FFBD00A614FF4FA304861C0
:106060008B61704770B50D4D04460A2809D10D218A
:106070002846FFF747FC80212846FFF74CFC002804
:10608000F9D0E1B22846FFF73DFC80212846FFF712
:1060900042FC0028F9D0204670BD000000380140C5
:1060A0004FF400518803FEF79FF8FEF717FC4FF4FA
:1060B000E120FFF79FFCFEF7E9F9FEF71DF92F48F5
:1060C000018B408BFDF706FBFEF7DEFFFCF7B6FB0E
:1060D0002BA0FFF70DFD002240F6FF714220FDF7D7
:1060E0003DFDFEF715F8FFF7ABF8FFF7BDFC4FF4E9
:1060F000FA70FDF7C5FAFDF7ABFAFFF7E9FCDFF838
:106100009080244D244C4FF480474FF4C8663946A4
:106110004046FDF79AFB78B100202070FEF77EFA2A
:10612000FEF782F82888B04217D21C480078012870
:1061300021D0FCF72BFEEAE720780A2801D2401C88
:106140002070C0B2052802D16078401C6070607871
:106150000428E3D101206070E0E7607840B10128B5
:1061600006D0022807D00328D1D1FCF757FACEE792
:10617000FCF724FBCBE7FCF7A1FAC8E7980F002057
:10618000737461727420696E69742069630A000017
:10619000003C0240A80000200000002080000020F9
:1061A0002DE9F04112484FF482770024858A0426B5
:1061B00039461048FBF7E3FF39460F48FBF7DFFF8E
:1061C0000D4F0C4B00223D801A8007EBC40003EBFF
:1061D000C40142804D8082808D80C580CA80641C4D
:1061E0000581E4B20A81B442EFD3BDE8F08100003A
:1061F000980F0020B6250020BA26002010B5034CC9
:106200002070A180E280238110BD0000C6290020FB
:1062100010B5034C20706170A270638110BD000046
:10622000C6290020273857388738B73827405740C5
:106230008740B740272857288728B7282730573066
:106240008730B7308710B7102710571027485748A6
:106250008748B748275057508750B75027185718C6
:106260008718B718272057208720B7202700570006
:106270008700B700270857088708B7082638563818
:106280008638B638264056408640B64026285628DE
:106290008628B628263056308630B6308610B6109E
:1062A00026105610264856488648B648265056505E
:1062B0008650B650261856188618B618262056202E
:1062C0008620B620260056008600B600260856080E
:1062D0008608B608253855388538B53825405540E4
:1062E0008540B540252855288528B52825305530C6
:1062F0008530B5308510B510251055102548554806
:106300008548B548255055508550B5502518551825
:106310008518B518252055208520B5202500550065
:106320008500B500250855088508B5082438543877
:106330008438B438244054408440B440242854283D
:106340008428B428243054308430B4308410B410FD
:1063500024105410244854488448B44824505450BD
:106360008450B450241854188418B418242054208D
:106370008420B420240054008400B400240854086D
:106380008408B408233853388338B3382340534043
:106390008340B340232853288328B3282330533025
:1063A0008330B3308310B310231053102348534865
:1063B0008348B348235053508350B3502318531885
:1063C0008318B318232053208320B32023005300C5
:1063D0008300B300230853088308B30822385238D7
:1063E0008238B238224052408240B240222852289D
:1063F0008228B228223052308230B2308210B2105D
:1064000022105210224852488248B248225052501C
:106410008250B250221852188218B21822205220EC
:106420008220B220220052008200B20022085208CC
:106430008208B208213851388138B13821405140A2
:106440008140B140212851288128B1282130513084
:106450008130B1308110B1102110511021485148C4
:106460008148B148215051508150B15021185118E4
:106470008118B118212051208120B1202100510024
:106480008100B100210851088108B1082038503836
:106490008038B038204050408040B04020285028FC
:1064A0008028B028203050308030B0308010B010BC
:1064B00020105010204850488048B048205050507C
:1064C0008050B050201850188018B018202050204C
:1064D0008020B020200050008000B000200850082C
:1064E0008008B008173847387738A7381740474032
:1064F0007740A740172847287728A7281730473024
:106500007730A7307710A710171047101748474863
:106510007748A748175047507750A7501718471883
:106520007718A718172047207720A72017004700C3
:106530007700A700170847087708A70816384638D5
:106540007638A638164046407640A640162846289B
:106550007628A628163046307630A6307610A6105B
:1065600016104610164846487648A648165046501B
:106570007650A650161846187618A61816204620EB
:106580007620A620160046007600A60016084608CB
:106590007608A608153845387538A53815404540A1
:1065A0007540A540152845287528A5281530453083
:1065B0007530A5307510A5101510451015484548C3
:1065C0007548A548155045507550A55015184518E3
:1065D0007518A518152045207520A5201500450023
:1065E0007500A500150845087508A5081438443835
:1065F0007438A438144044407440A44014284428FB
:106600007428A428143044307430A4307410A410BA
:1066100014104410144844487448A448145044507A
:106620007450A450141844187418A418142044204A
:106630007420A420140044007400A400140844082A
:106640007408A408133843387338A3381340434000
:106650007340A340132843287328A32813304330E2
:106660007330A3307310A310131043101348434822
:106670007348A348135043507350A3501318431842
:106680007318A318132043207320A3201300430082
:106690007300A300130843087308A3081238423894
:1066A0007238A238124042407240A240122842285A
:1066B0007228A228123042307230A2307210A2101A
:1066C00012104210124842487248A24812504250DA
:1066D0007250A250121842187218A21812204220AA
:1066E0007220A220120042007200A200120842088A
:1066F0007208A208113841387138A1381140414060
:106700007140A140112841287128A1281130413041
:106710007130A1307110A110111041101148414881
:106720007148A148115041507150A15011184118A1
:106730007118A118112041207120A12011004100E1
:106740007100A100110841087108A10810384038F3
:106750007038A038104040407040A04010284028B9
:106760007028A028103040307030A0307010A01079
:1067700010104010104840487048A0481050405039
:106780007050A050101840187018A0181020402009
:106790007020A020100040007000A00010084008E9
:1067A0007008A008073837386738973807403740EF
:1067B00067409740072837286728972807303730E1
:1067C0006730973067109710071037100748374821
:1067D0006748974807503750675097500718371841
:1067E0006718971807203720672097200700370081
:1067F0006700970007083708670897080638363893
:106800006638963806403640664096400628362858
:106810006628962806303630663096306610961018
:1068200006103610064836486648964806503650D8
:1068300066509650061836186618961806203620A8
:106840006620962006003600660096000608360888
:10685000660896080538353865389538054035405E
:106860006540954005283528652895280530353040
:106870006530953065109510051035100548354880
:1068800065489548055035506550955005183518A0
:1068900065189518052035206520952005003500E0
:1068A00065009500050835086508950804383438F2
:1068B00064389438044034406440944004283428B8
:1068C0006428942804303430643094306410941078
:1068D0000410341004483448644894480450345038
:1068E0006450945004183418641894180420342008
:1068F00064209420040034006400940004083408E8
:1069000064089408033833386338933803403340BD
:10691000634093400328332863289328033033309F
:1069200063309330631093100310331003483348DF
:1069300063489348035033506350935003183318FF
:10694000631893180320332063209320030033003F
:106950006300930003083308630893080238323851
:106960006238923802403240624092400228322817
:1069700062289228023032306230923062109210D7
:106980000210321002483248624892480250325097
:106990006250925002183218621892180220322067
:1069A0006220922002003200620092000208320847
:1069B000620892080138313861389138014031401D
:1069C00061409140012831286128912801303130FF
:1069D000613091306110911001103110014831483F
:1069E000614891480150315061509150011831185F
:1069F000611891180120312061209120010031009F
:106A000061009100010831086108910800383038B0
:106A10006038903800403040604090400028302876
:106A20006028902800303030603090306010901036
:106A300000103010004830486048904800503050F6
:106A400060509050001830186018901800203020C6
:106A500060209020000030006000900000083008A6
:106A6000600890084D4355566572040503055F03A1
:106A70002C18090000000000B71DC1046E3B8209FC
:106A8000D926430DDC7604136B6BC517B24D861AFD
:106A90000550471EB8ED08260FF0C922D6D68A2F1A
:106AA00061CB4B2B649B0C35D386CD310AA08E3C39
:106AB000BDBD4F3870DB114CC7C6D0481EE09345B2
:106AC000A9FD5241ACAD155F1BB0D45BC296975681
:106AD000758B5652C836196A7F2BD86EA60D9B63EC
:106AE00011105A6714401D79A35DDC7D7A7B9F707D
:106AF000CD665E74E0B6239857ABE29C8E8DA19173
:106B0000399060953CC0278B8BDDE68F52FBA582C8
:106B1000E5E66486585B2BBEEF46EABA3660A9B755
:106B2000817D68B3842D2FAD3330EEA9EA16ADA474
:106B30005D0B6CA0906D32D42770F3D0FE56B0DDA3
:106B4000494B71D94C1B36C7FB06F7C32220B4CE84
:106B5000953D75CA28803AF29F9DFBF646BBB8FB6F
:106B6000F1A679FFF4F63EE143EBFFE59ACDBCE8F0
:106B70002DD07DEC77708634C06D4730194B043DC5
:106B8000AE56C539AB0682271C1B4323C53D002EDC
:106B90007220C12ACF9D8E1278804F16A1A60C1BA1
:106BA00016BBCD1F13EB8A01A4F64B057DD0080858
:106BB000CACDC90C07AB9778B0B6567C69901571F1
:106BC000DE8DD475DBDD936B6CC0526FB5E6116260
:106BD00002FBD066BF469F5E085B5E5AD17D1D57A3
:106BE0006660DC5363309B4DD42D5A490D0B19441C
:106BF000BA16D84097C6A5AC20DB64A8F9FD27A536
:106C00004EE0E6A14BB0A1BFFCAD60BB258B23B627
:106C10009296E2B22F2BAD8A98366C8E41102F835C
:106C2000F60DEE87F35DA9994440689D9D662B9013
:106C30002A7BEA94E71DB4E0500075E4892636E922
:106C40003E3BF7ED3B6BB0F38C7671F7555032FA63
:106C5000E24DF3FE5FF0BCC6E8ED7DC231CB3ECF26
:106C600086D6FFCB8386B8D5349B79D1EDBD3ADC8F
:106C70005AA0FBD8EEE00C6959FDCD6D80DB8E602B
:106C800037C64F643296087A858BC97E5CAD8A73AD
:106C9000EBB04B77560D044FE110C54B38368646A6
:106CA0008F2B47428A7B005C3D66C158E440825589
:106CB000535D43519E3B1D252926DC21F0009F2C6E
:106CC000471D5E28424D1936F550D8322C769B3F31
:106CD0009B6B5A3B26D6150391CBD40748ED970AF8
:106CE000FFF0560EFAA011104DBDD014949B9319CD
:106CF0002386521D0E562FF1B94BEEF5606DADF89F
:106D0000D7706CFCD2202BE2653DEAE6BC1BA9EBF8
:106D10000B0668EFB6BB27D701A6E6D3D880A5DE61
:106D20006F9D64DA6ACD23C4DDD0E2C004F6A1CD44
:106D3000B3EB60C97E8D3EBDC990FFB910B6BCB43F
:106D4000A7AB7DB0A2FB3AAE15E6FBAACCC0B8A7B4
:106D50007BDD79A3C660369B717DF79FA85BB492FB
:106D60001F4675961A163288AD0BF38C742DB081C0
:106D7000C330718599908A5D2E8D4B59F7AB0854BD
:106D800040B6C95045E68E4EF2FB4F4A2BDD0C470C
:106D90009CC0CD43217D827B9660437F4F4600722D
:106DA000F85BC176FD0B86684A16476C9330046128
:106DB000242DC565E94B9B115E565A15877019182D
:106DC000306DD81C353D9F0282205E065B061D0B90
:106DD000EC1BDC0F51A69337E6BB52333F9D113EAF
:106DE0008880D03A8DD097243ACD5620E3EB152DEC
:106DF00054F6D4297926A9C5CE3B68C1171D2BCCE2
:106E0000A000EAC8A550ADD6124D6CD2CB6B2FDFD7
:106E10007C76EEDBC1CBA1E376D660E7AFF023EA68
:106E200018EDE2EE1DBDA5F0AAA064F4738627F963
:106E3000C49BE6FD09FDB889BEE0798D67C63A803E
:106E4000D0DBFB84D58BBC9A62967D9EBBB03E9313
:106E50000CADFF97B110B0AF060D71ABDF2B32A6B2
:106E60006836F3A26D66B4BCDA7B75B8035D36B5DF
:106E7000B440F7B100000000010203040102030462
:106E80000607080901020406080A0C102020202029
:106E900020202020010002000400060008000A0053
:106EA0000C001000200040008000000100010001E3
:106EB00000010001D46E000800000020E80000007E
:106EC000645B0008BC6F0008E8000020F02C0000A4
:106ED000745B0008000000000100000001000000D9
:106EE00000007900330000000000000000000001F5
:106EF00002050607080A0B0C0F000E06F505DC0557
:106F0000C305AA05910578055F0546052D051405FD
:106F1000FB04E204C904B00497047E0465044C0435
:106F200033041A040104E803CF03B6039D0384036A
:106F30006B03520339032003070300010203040516
:106F400006070E0F00000000000000000000000017
:106F50000000000000001100000FFF000000000012
:106F60000000000000000000000000000000000021
:106F70000000000000000000000000000000000011
:106F800000000F001E002D003C004B005A0069005D
:106F9000780087009600A500B400C300D200E1008D
:106FA000F000FF000E011D012C013B014A015901B7
:0C6FB000680100000020A10700000000A4
:0400000508002115B9
:00000001FF
